:020000040000FA
:040000006F303A28FB
:08000800A000030EA100831209
:1000100005191028831601178312B23081002B288E
:1000200083160113831203140B190310A80DA90DD5
:10003000AA0DAB0DAC0DAC16FF302C02031D2B2806
:10004000FA302B02031D2B2831152A08AF0029088E
:10005000AE002808AD008B100B11210E8300A00EFE
:04006000200E090065
:0C007400203084008001840A6030040207
:10008000031C3C281230B0008F218316FF23900000
:10009000831283160C308505870183128501870141
:1000A000073099000030831691008312C830831600
:1000B0008100831231309000003083168C0083124F
:1000C00010308B00831600309B001C141A0883121A
:1000D000BC00831610309B001C141A088312BD004C
:1000E000BD21831620309B001C141A088312C20005
:1000F0000130C2080319C20081018E018F010B116A
:100100008B100B108C018B179420311997207321C1
:10011000B30B9228031085190314B90DF03039027E
:1001200003191C21BE2184286400321008003111FB
:100130000130B7008B132030370783169B001C1447
:100140001A088312A4001030370783169B001C1472
:100150001A088312A300A6000230A6060030370753
:1001600083169B001C141A088312A200A7000130FA
:10017000A7068B17321CC22822090339A200A30943
:10018000A409A50924082F02031D162923082E02FD
:10019000031D162922082D02031D162901303702DE
:1001A000031DD7283D18D7283D143E149621023050
:1001B0003702031DE028BD18E028BD143E149F211E
:1001C00003303702031DE9283D19E9283D153E1487
:1001D000A82104303702031DF228BD19F228BD15ED
:1001E0003E14B12105303702031DFB283D1AFB28C0
:1001F0003D163E14B92106303702031D0429BD1AED
:100200000429BD163E14BA2107303702031D0D29FB
:100210003D1B0D293D173E14BB2108303702031D3D
:100220001629BD1B1629BD173E14BC21B70A05307F
:100230003702031808009A280130B600B300B40052
:10024000B500B70085018701B1139420B30B422993
:10025000031085190314B90DF03039020319692907
:10026000B41F8501B41F8701B40B42293708B608B3
:100270000319B60003194029FF3085008700B60333
:100280009630B400311D25293111321C4C292D091D
:100290000339AD00AE09AF092F1C25298E018F014E
:1002A0000C1C25290C102E1E25298B1320303707F6
:1002B000BB002F08BA007C2110303707BB002E0886
:1002C000BA007C2100303707BB002D08BA007C2122
:1002D0008B1785018701B70AB60105303702031C69
:1002E0002529BD2108003E1C08003E101030BB002F
:1002F0003D08BA007C2108008B133A0883161C15B0
:100300009A003B089B0055309D00AA309D009C142C
:1003100064009C1888291C1183128B170800013077
:10032000D500D200EE30D000D10008000130D50059
:10033000D200EE30D000D1000130BD000800013005
:10034000D500D200EE30D000D1000230BD00080050
:100350000130D500D200EE30D000D1000430BD0015
:1003600008000130D500D200EE30D000D100BD0130
:100370000800080008000800080008008F0803199A
:1003800008008F01C10B08004208C100D50B08000E
:100390005608D50007303D050319F529D21BD00AB0
:1003A000D21FD0030A305002031CF029D0010930BB
:1003B000D21FD0005203D2007F39031DF029D10A89
:1003C00010305102031CE529D1015022D2006022D5
:1003D000D4007022D600D500D0010930D21FD00041
:1003E0000023850024238700080085018701080079
:1004A00002308A0051083D1C572A883E8200BD1C3C
:1004B0005B2A883E82003D1D5F2A983E8200003400
:1004C00002308A0051083D1C672AA83E8200BD1CEC
:1004D0006B2AB83E82003D1D6F2AB83E8200003470
:1004E00002308A0051083D1C772AC83E8200BD1C9C
:1004F0007B2AD83E82003D1D7F2AE83E82000134DF
:100510000734873407348734033483340334833413
:100520000B3403340F3407340B34033403340734EF
:10053000053487340734253483340334073489344D
:100540000B3403348F3405348B34113403340334C7
:1005500001340134023402340434043408340834DD
:10056000103410342034203440344034803480340B
:10057000083404340234803440348034103402347B
:10058000043410342034013404344034843480344E
:10059000093409340A340A34083408340834083475
:1005A0000834183408341834083418341034083433
:1005B000093429340A341A34283408340834083405
:1005C0000A34383408341A3408345834103448346F
:1005D000293409340A340A342834083408344834B5
:1005E0002834183488341834283418341034083433
:1006000003308A005008541C072B4B3E8200D41C38
:100610000B2B563E8200541D0F2B613E8200D41DD1
:10062000132B6C3E8200541E172B773E8200D41E83
:100630001B2B823E8200541F1F2B8D3E8200D41F35
:10064000232B983E8200003403308A005008541C4B
:100650002B2BA33E8200D41C2F2BAE3E8200541DB8
:10066000332BB93E8200D41D372BC43E8200541E6A
:100670003B2BCF3E8200D41E3F2BDA3E8200541F1C
:10068000432BE53E8200D41F472BF03E820000340E
:0A0696001034203401340234003423
:0A06A000003400340034003400344C
:0406AC0010343034A2
:1006B0003134333433343334333433343334333404
:0E06C2000034003400340034003400340234BC
:0606D0000334233433342F
:0806D800103420340134023417
:0C06E000003410342034013402340034A3
:0206EE001034C6
:1006F0002034013402340034003402340134203414
:020700001034B3
:0C070400103430343134333433343334A7
:080710003134303410340034A0
:06071A00333423340334E4
:0E072000023400340034023403342334333402
:10073000333400343334003433340034333400344D
:04074000333400341A
:0A07460000340034003400340234A3
:0A075000043401342034103408345E
:04075C000034003431
:1007600000340034023406340734273437343F343D
:0E07720008341834383439343D343F343F34C1
:060780003F343F343F341A
:08078800043401342034103464
:0C0790000A3404340134203410340A34DC
:02079E0008341D
:1007A000103420340134063406340134203410343B
:0207B00008340B
:0C07B40008341834383439343F343934F8
:0807C000383418340834003409
:0607CA003F3437342734F0
:0E07D0000734063406340734273437343F34F8
:1007E0003F3400343F3400343F3400343F3400346D
:0407F0003F3400345E
:084000000C00030002000600A1
:02400E00CC01E3
:10420000010078007A007C007E007B0079007F004E
:104210007D007A0078007E007C00FF00FF00FF0038
:104220000000F200F600FA00FE00F200F600FA00CC
:10423000FE00F200F600FA00FE00FF00FF00FF00A3
:10424000010005000500050005000900090009003E
:1042500009000D000D000D000D00FF00FF00FF0024
:10426000FF00FF00FF00FF00FF00FF00FF00FF0056
:10427000FF00FF00FF00FF00FF00FF00FF00FF0046
:10428000FF00FF00FF00FF00FF00FF00FF00FF0036
:10429000FF00FF00FF00FF00FF00FF00FF00FF0026
:1042A000FF00FF00FF00FF00FF00FF00FF00FF0016
:1042B000FF00FF00FF00FF00FF00FF00FF00FF0006
:1042C000FF00FF00FF00FF00FF00FF00FF00FF00F6
:1042D000FF00FF00FF00FF00FF00FF00FF00FF00E6
:1042E000FF00FF00FF00FF00FF00FF00FF00FF00D6
:1042F000FF00FF00FF00FF00FF00FF00FF00DD00E8
:00000001FF
